S01E000062696E2F64656D6F70726F675F73746D3332663039312E7372656329
S315080028000080002085290008D7290008D929000852
S3150800281000000000000000000000000000000000AA
S31508002820000000000000000000000000DB2900088E
S315080028300000000000000000DD290008C54000086F
S31508002840E3290008E5290008E7290008E92900081E
S31508002850EB290008ED290008EF290008F1290008EE
S31508002860F3290008F5290008F7290008F9290008BE
S31508002870FB290008FD290008FF290008012A00088D
S31508002880032A0008052A0008072A0008092A00085A
S315080028900B2A00080D2A00080F2A0008112A00082A
S315080028A0132A0008152A0008172A0008192A0008FA
S315080028B01B2A00081D2A00081F2A0008212A0008CA
S315080028C0EE11AA5510B5064C2378002B07D1054BF7
S315080028D0002B02D0044800E000BF0123237010BD7E
S315080028E02C01002000000000A4460008044B10B587
S315080028F0002B03D00349044800E000BF10BDC046C2
S315080029000000000030010020A4460008164B002BEA
S3150800291000D1144B9D46402292029A1A92460021F3
S315080029208B460F461348144A121A01F077FE0F4BCE
S31508002930002B00D098470E4B002B00D0984700205C
S31508002940002104000D000D48002802D00C4800E0C4
S3150800295000BF01F03FFE2000290001F0E9FB01F06D
S3150800296023FEC0460000080000800020000000008A
S31508002970000000002C0100203402002000000000A6
S315080029800000000008498D460849094A094B9B1A68
S3150800299005DD00240859105104349C42FADB064828
S315080029A0804706480047000000800020B04600081F
S315080029B0C00000202C0100202D2A00080D2900083F
S315080029C01849194A002301E00B6004319142FBD3F0
S315080029D001F0AEFBFEE7FEE7FEE7FEE7FEE7FEE7F1
S315080029E0FEE7FEE7FEE7FEE7FEE7FEE7FEE7FEE7B1
S315080029F0FEE7FEE7FEE7FEE7FEE7FEE7FEE7FEE7A1
S31508002A00FEE7FEE7FEE7FEE7FEE7FEE7FEE7FEE790
S31508002A10FEE7FEE7FEE7FEE7FEE7FEE7FEE7FEE780
S31508002A20FEE7FEE72C01002034020020114B1A684D
S31508002A3001210A431A605A680F4802405A601A6808
S31508002A400E4802401A601A680D4802401A605A6811
S31508002A500C4802405A60DA6A0F208243DA621A6B1F
S31508002A60094802401A635A6B8A435A6300229A60DD
S31508002A707047C046001002400CB8FF08FFFFF6FE7C
S31508002A80FFFFFBFFFFFFC0FFACFEF0FFF0B5CE4631
S31508002A90474680B583B004000368DB072BD5BD4BDA
S31508002AA05A680C231340042B1DD0BA4B5A680C23C2
S31508002AB01340082B0ED06368012B43D0002B5AD144
S31508002AC0B44B1A68B4490A401A601A68B3490A40EE
S31508002AD01A603DE0AF4B5B68C02252021340802269
S31508002AE052029342E7D1AB4B1B689B0303D563683D
S31508002AF0002B00D15BE223689B077DD5A54B5B685D
S31508002B000C221A4268D0A34B5A680C231340082B90
S31508002B1059D0E368002B00D195E09E4A136801213D
S31508002B200B43136001F0FAF907009A4E0225336841
S31508002B301D4200D07EE001F0F1F9C01B0228F6D94B
S31508002B40032072E0934A116880235B020B431360EB
S31508002B506368002B27D001F0E1F907008D4E802528
S31508002B60AD0233682B42C6D101F0D8F9C01B6428E0
S31508002B70F7D9032059E0052B09D0864B1A688649F0
S31508002B800A401A601A6885490A401A60E0E7814BCC
S31508002B9019688022D2020A431A60196880225202F2
S31508002BA00A431A60D4E701F0B9F90700794E80257F
S31508002BB0AD0233682B429ED001F0B0F9C01B6428E1
S31508002BC0F7D9032031E0734B5B68C02252021340E9
S31508002BD08022120293429CD16E4B1B689B0703D539
S31508002BE00120E368012B20D16A490A682369DB00C2
S31508002BF0F820824313430B6023681B074BD5E36910
S31508002C00002B34D0634A536A01210B43536201F007
S31508002C1085F907005F4E0225736A1D423BD101F014
S31508002C207DF9C01B0228F7D9032003B00CBC9046D7
S31508002C309946F0BD57490A682369DB00F8208243A4
S31508002C4013430B60D8E7534A136801218B4313607B
S31508002C5001F064F907004F4E022533681D42CBD0B8
S31508002C6001F05CF9C01B0228F7D90320DDE7494AC1
S31508002C70536A01218B43536201F050F90700454E10
S31508002C800225736A1D4206D001F048F9C01B0228C6
S31508002C90F7D90320C9E723685B0700D487E03D4BD3
S31508002CA0DB6900229046DB000BD43A4AD1698020C2
S31508002CB040050143D161D36903400193019B012378
S31508002CC09846374B1B68DB050ED5A368012B21D028
S31508002CD0002B38D12F4B1A6A01218A431A621A6AC5
S31508002CE003318A431A621AE02D4A116880235B0071
S31508002CF00B43136001F012F90500294F8026760070
S31508002D003B683342E1D101F009F9401B6428F7D941
S31508002D1003208AE71F4A136A01210B431362A3683B
S31508002D20002B26D001F0FAF881461A4F02261D4DCF
S31508002D303B6A1E4238D101F0F1F84B46C01AA84248
S31508002D40F6D9032071E7052B09D0124B1A6A01211F
S31508002D508A431A621A6A03318A431A62DFE70D4BFD
S31508002D601A6A04210A431A621A6A03390A431A625A
S31508002D70D5E701F0D3F88146064F0226094D3B6A8E
S31508002D801E4211D001F0CAF84B46C01AA842F6D91D
S31508002D9003204AE700100240FFFFFEFFFFFFFBFF8C
S31508002DA000700040881300004346012B3CD023687E
S31508002DB0DB0610D56369012B3CD005335BD17E4A0F
S31508002DC0536B04218B435363516BA369DB00F820D3
S31508002DD081430B43536323689B0674D5764B5A6825
S31508002DE00C2313400C2B65D0734B5A680C231340E5
S31508002DF0082B58D0236A002B00D186E06E4A516B07
S31508002E0080235B020B43536301F088F807006A4E80
S31508002E1080256D02736B2B4255D101F07FF8C01BDC
S31508002E200228F7D9032000E7634AD36963490B40B0
S31508002E30D361BCE7604B5A6B04210A435A635A6B49
S31508002E4003390A435A6301F069F807005A4E022506
S31508002E50736B1D4206D101F061F8C01B0228F7D931
S31508002E600320E2E654494A6BA369DB00F820824353
S31508002E7013434B63AFE7504B5A6B04210A435A631B
S31508002E805A6B03398A435A6301F048F807004A4ED9
S31508002E900225736B1D429ED001F040F8C01B022824
S31508002EA0F7D90320C1E6444B5B68C022520213409F
S31508002EB093429FD1404B5B6BDB0304D50120236A09
S31508002EC0012B00D0B1E6636A0020002B00D1ACE6E6
S31508002ED0394A51680C220A40082A6AD0022B29D09E
S31508002EE0354A136836490B40136001F017F8060097
S31508002EF0314D8024A4042B68234256D001F00EF8E5
S31508002F00801B0228F7D903208FE62B4A536B2D49DD
S31508002F100B40536301F002F80700274E80256D0227
S31508002F20736B2B42CFD000F0F9FFC01B0228F7D9EC
S31508002F3003207AE6204A136821490B40136000F003
S31508002F40EDFF07001C4E8025AD0433682B4206D0E2
S31508002F5000F0E4FFC01B0228F7D9032065E6164BEC
S31508002F60DA6A0F218A43216B0A43DA625968E26AF0
S31508002F70A06A0243144801400A435A60196880222D
S31508002F8052040A431A6000F0C9FF06000A4D80245D
S31508002F90A4042B68234206D100F0C0FF801B022838
S31508002FA0F7D9032041E600203FE600203DE6012050
S31508002FB03BE6012039E6C04600100240FFFFFFEF5E
S31508002FC0FFFFFFFEFFFFFEFFFF7FC2FF30B589B0A0
S31508002FD004AA214B180032C832C2110002680A60DE
S31508002FE06A46103313CB13C21B6813601B4B5B680E
S31508002FF00C20184008280AD00C3843425841404251
S31508003000174B1840174B9C46604409B030BD990CC5
S315080030100F22114004A8445C1049C96A0A4069464F
S31508003020895CC0225202134080225202934208D081
S31508003030C0225202934209D00A4801F029FA604395
S31508003040E3E7084801F024FA6043DEE7064801F0A2
S315080030501FFA6043D9E7C0465C46000800100240E4
S31508003060005A620200127A00006CDC02F8B5CE46FD
S31508003070474680B504000D005F4B1A6801231340CC
S315080030808B420BD25C490B68012293432B430B609E
S315080030900B681A400120AA4200D0A7E023689B07C4
S315080030A006D5564A5368F0218B43A1680B435360F3
S315080030B02368DB0770D56268012A09D0022A2CD05A
S315080030C0032A30D04D4B1B689B0706D401208DE0A0
S315080030D04A4B1B689B0300D48CE048494B68032085
S315080030E0834313434B6000F019FF06006368012B06
S315080030F01FD0022B2ED0032B3DD0404B98460C27D1
S315080031003F4B994643465B681F4245D000F006FF91
S31508003110801B4845F6D9032068E0384B1B689B019D
S31508003120DBD4012062E0354B5B6BDB03D5D4012091
S315080031305CE0324B98460C27314B994643465B6810
S315080031403B40042B28D000F0E9FE801B4845F5D902
S3150800315003204BE0294B98460C27294B99464346B2
S315080031605B683B40082B17D000F0D8FE801B48450B
S31508003170F5D903203AE0214B98460C27204B99466F
S3150800318043465B683B400C2B06D000F0C7FE801B0D
S315080031904845F5D9032029E0174B1A68012313403F
S315080031A0AB420AD914490B68012293432B430B609F
S315080031B00B681A400120AA4218D123685B0706D576
S315080031C00E4A53680F490B40E1680B435360FFF7FB
S315080031D0FDFE0A4B5B681B061B0F0B4AD35CD840E7
S315080031E00A4B1860002000F06FFE00200CBC9046C9
S315080031F09946F8BD0120F9E7002002400010024078
S3150800320088130000FFF8FFFF44460008C0000020AE
S31508003210014B18687047C046C0000020044B5B6825
S315080032205B055B0F034AD35C034A1068D8407047B6
S315080032300010024054460008C0000020704770B5D0
S31508003240041E00D1A2E02023C35C002B1BD02268F9
S31508003250136802218B43136000F060FE0600022506
S3150800326023685A68154211D000F058FE801B0A28B8
S31508003270F6D9626A80239B021343636220230522E0
S31508003280E254012070BDFFF7D9FFE0E71A68012173
S315080032900A431A6000F042FE0600012523685A68B0
S315080032A015420ED100F03AFE801B0A28F6D9626A4A
S315080032B080239B021343636220230522E2540120E4
S315080032C0E0E7227E012A3ED01A6880218A431A60E6
S315080032D0637E012B3CD02268136840218B43136020
S315080032E0A37E012B3AD02268136820218B431360F2
S315080032F0E37E012B38D02268136810210B43136034
S31508003300237F012B36D02268136808218B4313606C
S31508003310637F012B34D02268136804218B43136022
S315080033202168A368E2681343226913436269134359
S315080033306268013A1343CB6100236362203301229A
S31508003340E25400209EE71A6880210A431A60BFE704
S315080033502268136840210B431360C1E7226813688B
S3150800336020210B431360C3E72268136810218B439F
S315080033701360C5E72268136808210B431360C7E783
S315080033802268136804210B431360C9E7012079E713
S3150800339030B52023C35C013B012B06D9426A802342
S315080033A0DB0213434362012030BD03688024A40076
S315080033B018590122104318511F204C692040824099
S315080033C08725AD005859D44320405851C86900286C
S315080033D014D1103D585920405851C86805048888AA
S315080033E0054348694830C000C55088680504088800
S315080033F0054348694830C00018184560C86901285F
S315080034001AD0886900282ED18125AD005859204048
S315080034105851086900282CD18525AD005859044013
S315080034205C51096A01292AD0802189005A5801204D
S3150800343082435A500020B7E78325AD0058591043F8
S315080034405851086805048888054348694830C0000B
S31508003450C550886805048889054348694830C0000E
S3150800346018184560CDE78125AD00585910435851C5
S31508003470CFE78524A400185910431851D1E78720AF
S31508003480800019580A431A50CEE770B50400202365
S31508003490C35C012B06D0426A80231B031343436295
S315080034A0012070BD1F330222C2540268136801212D
S315080034B08B43136000F032FD0600012523685B6824
S315080034C01D420ED000F02AFD801B0A28F6D9626A32
S315080034D080239B021343636220230522E2540120C2
S315080034E0DFE7002363620020DBE770B52024045D74
S315080034F0013C012C00D991E000290AD10468E4684E
S31508003500A40711D1426A80239B0313434362012017
S315080035108AE004682469A40706D1426A80239B03CB
S315080035201343436201207FE00C001B342401056825
S31508003530655904242C40946061D10C001B34240185
S3150800354005686459640D14600C001B342401056871
S315080035506559AD07ED0FD56005682D196E680F25FD
S315080035603540156105682D196D682D042D0E956178
S315080035700568AC4664446468240C54610A0104680E
S31508003580A418B934FF3424681C700468A418B93424
S31508003590FF342468240A5C700468A418B934FF341C
S315080035A02468240C9C700468A418B934FF34246871
S315080035B0240EDC700468A418BD34FF3424681C711A
S315080035C00468A418BD34FF342468240A5C710468AE
S315080035D0A418BD34FF342468240C9C710468A446DE
S315080035E06244BD32FF321268120EDA7100290ED11A
S315080035F00268D36820310B43D360002014E00C0026
S315080036001B34240105686459E40854609CE7026881
S31508003610136920210B431361002005E0426A8023C9
S31508003620DB0213434362012070BD000070B5002819
S3150800363014DB8408A400144B9C466444C026B600D8
S31508003640A55903221040C000FF231A008240954363
S3150800365089010B4083401D43A55170BDC0B20F229E
S315080036600240083A92089200084BD318DD690324F1
S315080036702040C000FF2214008440A54389010A4067
S3150800368082402A43DA61E8E700E100E000ED00E065
S3150800369001380A4B98420FD8094A50600948036A0C
S315080036A01B021B0AC02109060B4303620023936011
S315080036B007331360002070470120FCE7FFFFFF0077
S315080036C010E000E000ED00E0042805D0054A136884
S315080036D004218B4313607047024A136804210B4385
S315080036E01360F8E710E000E0704710B5FFF7FCFF3D
S315080036F010BD0000F0B5DE4657464E464546E0B5D5
S3150800370085B00A68002A00D1BDE000230124A4463A
S315080037100F34A2460D3CA14680246405A3465D4CA1
S315080037200419651EAC41043401943AE0DC08A4008F
S315080037300419276A07251D40AD000F22AA409743A2
S315080037400A69AA4015003D43256234E00025B540C4
S315080037503D43A560504C2468009AD5434A68D20375
S3150800376000D584E02C404C4E346074684A68920355
S3150800377000D57FE02C40484E7460B4684A68D2028F
S315080037807BD42C40444EB460F4684A68920277D4DD
S3150800379022002A40404CE26001330A681400DC40EB
S315080037A071D066469E4032400092F5D04C68554628
S315080037B0AC43022CBAD004685F004D46BD40ED43C9
S315080037C02C40A0464C684A461440BC404246144326
S315080037D004604C6852469443013C012C11D8846815
S315080037E02C40A046CC68BC404246144384604468DA
S315080037F0B44326004A681409624614409C40344380
S315080038004460C4682C408D68BD402543C5604A683D
S315080038105C462242C0D0214CA56962461543A56183
S31508003820A46914400394039C9C08A4001C4A90466F
S315080038304444A5684E461E40B6000F27B740BD4310
S315080038402F009025ED05A84200D17FE7154DA84227
S3150800385007D0154DA84206D0144DA84205D0019DA3
S3150800386075E7654673E7022571E74D466FE7009AE7
S31508003870144378E7009A14437DE7009A144381E7D6
S31508003880009A224386E705B03CBC90469946A24674
S31508003890AB46F0BD00F0FFB700040140001002403F
S315080038A0000001400004004800080048000C0048D9
S315080038B0002A01D0816170478162FCE770470000E9
S315080038C070B5040001680A68836800690343606983
S315080038D00343E06903438A48024013430B602268A6
S315080038E0536888490B40E1680B43536021688A682E
S315080038F0A369206A03438448024013438B60256802
S31508003900824B9D4222D0824B9D4235D0814B9D42AF
S3150800391000D172E0804B9D4200D199E07F4B9D42D9
S3150800392000D195E07E4B9D4200D191E07D4B9D42B2
S3150800393000D18DE07C4B9D4200D189E080231B029B
S31508003940E2699A4200D17DE0012055E0774B1A6B77
S3150800395003231340012B00D1AEE0002B33D0022BFA
S3150800396000D1BBE0032B1BD080231B02E2699A42DD
S3150800397000D16AE001203FE06C4B1B6BC02292022B
S31508003980134080225202934200D195E019D9802231
S315080039909202934200D1A1E0C02292029342E3D15F
S315080039A080231B02E2699A423ED061684808604B50
S315080039B09C46604400F06CFD0004000CE8600020A2
S315080039C01AE0002BD0D180231B02E2699A4244D127
S315080039D0FFF724FC400063685B08C018616800F0C4
S315080039E057FD83B200200F22190091430A0021686F
S315080039F01B075B0F1343CB6070BD4C4B1B6BC02280
S31508003A00120313408022D202934233D017D9802260
S31508003A10120393423FD0C02212039342A4D18023BB
S31508003A201B02E2699A42C0D163685808414B9C461A
S31508003A306044616800F02CFD83B20020D3E7002BB8
S31508003A40C1D091E701200023CDE701200023CAE772
S31508003A5080231B02E2699A42BAD0FFF7DFFB61684E
S31508003A6024684B08181800F013FD0004000CE060E9
S31508003A700020C1E780231B02E2699A4221D1FFF7A1
S31508003A80A5FA400063685B08C018616800F000FD8D
S31508003A9083B20020A7E780231B02E2699A4222D15B
S31508003AA06368580880235B029C466044616800F09E
S31508003AB0EFFC83B2002096E780231B02E2699A4254
S31508003AC0DDD0FFF783FA616824684B08181800F000
S31508003AD0DFFC0004000CE06000208DE780231B0259
S31508003AE0E2699A42DCD06168480880231B029C463A
S31508003AF0604400F0CDFC0004000CE86000207BE781
S31508003B00F369FFEFFFCFFFFFFFF4FFFF0038014027
S31508003B100044004000480040004C0040005000406F
S31508003B200014014000180140001C0140001002402A
S31508003B3000127A000024F400436ADB0706D50268FF
S31508003B4053682C490B40816A0B435360436A9B07B1
S31508003B5006D50268536828490B40C16A0B4353606F
S31508003B60436A5B0706D50268536824490B40016B14
S31508003B700B435360436A1B0706D5026853682049FE
S31508003B800B40416B0B435360436ADB0606D502685C
S31508003B9093681C490B40816B0B439360436A9B06F1
S31508003BA006D50268936818490B40C16B0B439360AE
S31508003BB0436A5B060BD50268536814490B40016CCF
S31508003BC00B43536080235B03026C9A420AD0436A14
S31508003BD01B0606D5026853680D490B40816C0B43DA
S31508003BE053607047026853680A490B40416C0B439F
S31508003BF05360ECE7FFFFFDFFFFFFFEFFFFFFFBFF44
S31508003C00FF7FFFFFFFEFFFFFFFDFFFFFFFFFEFFF76
S31508003C10FFFFF7FFFFFF9FFFF0B5C64600B5070099
S31508003C200C0016009846069D3A68D36923401B1B6C
S31508003C3059424B41B3421ED16B1CF6D0002D05D01C
S31508003C4000F06CF94346C01AA842EDD93A681368E1
S31508003C500B490B4013603A689368A331FF318B43D5
S31508003C60936020236922BB540132BB544833002297
S31508003C70FA54032000E0002004BC9046F0BDC0467C
S31508003C805FFEFFFFF0B5D646474680B585B004000F
S31508003C900D00170098466A23C35C202B00D085E0E8
S31508003CA0002900D188E0002A00D187E080235B0143
S31508003CB082689A4221D06823E35C012B00D17FE019
S31508003CC068230122E2540023E3666A332132E25470
S31508003CD000F024F903905823E7520233E752A36809
S31508003CE08022520193420FD0002B1CD12369002B4E
S31508003CF015D15C33FF22E25219E00369002BDAD1B1
S31508003D00CB07D8D5012052E02369002B03D15C33B9
S31508003D102D4AE2520BE05C23FF22E25207E05C23C5
S31508003D207F22E25203E080225205934206D05C23AA
S31508003D30E35A9A465A278026760110E02369002B13
S31508003D4003D15C337F22E252F1E75C233F22E25241
S31508003D50EDE723689B8C524613402B700135E35BD5
S31508003D609BB2002B1AD0E35B013B9BB2E35343465D
S31508003D700093039B002220212000FFF74DFF002817
S31508003D8020D1A368B342E4D12369002BE1D123688B
S31508003D909B8C524613402B800235E0E76A3320227B
S31508003DA0E254023B0022E254002000E0022005B063
S31508003DB00CBC90469A46F0BD0120F8E70120F6E7CC
S31508003DC00220F4E70320F2E7FF01000030B583B0D4
S31508003DD004000023C36600F0A1F8050023681A4A08
S31508003DE0934205D0194A934202D0194A934206D102
S31508003DF01B681B070ED423681B685B0717D4202390
S31508003E006922A3540132A35448330022E254002005
S31508003E1003B030BD80210F4B00932B00002289038D
S31508003E202000FFF7F9FE0028E5D00320F0E78021FF
S31508003E30084B00932B000022C9032000FFF7ECFE75
S31508003E400028DCD00320E3E70038014000440040A6
S31508003E5000480040FFFFFF0110B5041E30D069235B
S31508003E60C35C002B22D069232422E25422681368FB
S31508003E7001218B4313602000FFF722FD012814D08F
S31508003E80636A002B18D1226853680E490B405360A9
S31508003E90226893682A218B4393602268136829391C
S31508003EA00B4313602000FFF791FF10BD6833002213
S31508003EB0C254FFF703FDD6E72000FFF73DFEE2E711
S31508003EC00120F2E7FFB7FFFF10B50400FFF7A0F9DE
S31508003ED0FA21890000F0DCFAFFF7DAFB012000225C
S31508003EE021004042FFF7A2FB002010BD10B5064A8C
S31508003EF0136810210B4313600020FFF7E5FF00F05D
S31508003F0051F9002010BDC04600200240024A13683D
S31508003F10013313607047C04630020020014B186811
S31508003F207047C04630020020F0B5CE46474680B5F9
S31508003F3083B004000368DB0336D54E4BDB690025E6
S31508003F40DB000AD44B4AD169802040050143D16180
S31508003F50D36903400193019B0135474B1B68DB0579
S31508003F605AD5444B1B6AC0229200134013D061688D
S31508003F700A409A420FD03F4B186A404A02401E6ACE
S31508003F808021490231431962196A3D4E314019624E
S31508003F901A62C30757D4374A136A38490B4061680F
S31508003FA00B431362012D60D02368DB0706D5314A1F
S31508003FB0136B03218B43A1680B43136323689B0789
S31508003FC006D52C4A136B2F490B40E1680B43136344
S31508003FD023685B0306D5274A136B2B490B402169D7
S31508003FE00B43136323689B0606D5224A136B1021DD
S31508003FF08B4361690B431363002023685B0506D571
S315080040001C4A136B40218B43A1690B43136303B00E
S315080040100CBC90469946F0BD174A116880235B0090
S315080040200B431360FFF77AFF8046134F802676000E
S315080040303B68334295D1FFF771FF4346C01A64289F
S31508004040F6D90320E3E7FFF769FF8146094F022601
S315080040500E4B98463B6A1E429DD1FFF75FFF4B46C3
S31508004060C01A4045F6D90320D1E7D36908490B4061
S31508004070D36199E70010024000700040FFFCFFFF83
S31508004080FFFFFEFFFFFFFCFFFFFFF3FF88130000A3
S31508004090FFFFFFEFFEE710B5FFF7BAF8FA21890030
S315080040A000F0F6F9FFF7F4FA0420FFF70DFB0120FC
S315080040B0002200214042FFF7B9FA10BD10B5FFF7FC
S315080040C02DFF10BD10B5FFF721FFFFF70EFB10BD42
S315080040D010B5902000222021C005FFF7E9FB10BD8E
S315080040E010B5FFF7EBFF04000F4B1B68C31AF42249
S315080040F0FF3293420ED90D4B1B78002B0BD10B4B7D
S31508004100F33AFF3A1A7090202021C005FFF7D0FB3A
S31508004110054B1C6010BD054B00221A70902020210B
S31508004120C005FFF7C5FBF3E74C0100204801002056
S3150800413000B599B0FFF7DAFE01230B9305220C921E
S31508004140033A1492802252021592A02292031692E2
S3150800415017930BA8FEF79AFC002800D0FEE7072362
S315080041600093053B019300230293039301216846BC
S31508004170FEF77CFF002800D0FEE702230493002305
S31508004180079304A8FFF7D0FE002800D0FEE7FFF744
S315080041909FFFFFF780FF00F06FF8FFF7A1FF00F021
S315080041A007F9FAE7F0B58BB0314B9A6901252A432E
S315080041B09A619A692A400092009A59698022920265
S315080041C0114359615969114001910199586980242F
S315080041D0E402204358615969214002910299D9693C
S315080041E01143D961D9690A400392039ADA69802191
S315080041F089040A43DA61DB690B400493049B0520B2
S31508004200002200214042FFF711FA02200022002175
S315080042104042FFF70BFA0120002200214042FFF737
S3150800422005FA2023059306950024079408949027F9
S31508004230FF0505A93800FFF75DFA0C23059302264A
S31508004240069607940894099505A93800FFF752FAC7
S31508004250C0239B000593069607940323089301330E
S31508004260099305A90348FFF745FA0BB0F0BDC04608
S315080042700010024000040048F0B5DE464F464646A8
S31508004280C0B58CB03B483C4B0360E1231B0243603E
S3150800429000238360C36003610C2242618361C361AA
S315080042A003624362FFF7D8FDFEF7B8FFFA218900DB
S315080042B000F0EEF80190314D24239B46AB440023D1
S315080042C099462F4B984602E002355D4519D02F785E
S315080042D06E78BA1901325401A41AA400A418A400CD
S315080042E02100019800F05AF90029EDD12100019822
S315080042F000F0CEF883B29946013B9BB24345E3D81A
S3150800430001E0002600271F4C1F4B23600025257659
S315080043106576A57601239846E37625776577A560C1
S31508004320E560013F3F042761013E360566614B465D
S3150800433063602000FEF783FF0795089543460993B7
S31508004340124B02930395124B049304230593069587
S3150800435043460A930D330B9302A92000FFF718F87A
S315080043602000FFF792F80CB01CBC90469946A3466D
S31508004370F0BDC04678010020004400407C46000895
S31508004380FF0300005001002000640040E0CC00005C
S31508004390E0FF0000BFF34F8F034B044ADA60BFF318
S315080043A04F8FC046FDE7C04600ED00E00400FA0561
S315080043B000B58BB02F4B1B78002B24D101222E4938
S315080043C02E48FFF75FFC00280DD001AB03AA002199
S315080043D02B48FFF78AF8002803D12A4B039A9A42FA
S315080043E03CD00BB000BD244B1B78013B3F2BECD8CF
S315080043F0FFF764FE244B18601E4B01221A70234BEC
S3150800440000221A70E1E7214B1B7801331A49C918B3
S31508004410002301221948FFF735FC002813D11B4A4F
S3150800442013780133DBB21370134A12789A42CCD14F
S31508004430104A00211170104A5278FF2AC5D1022B62
S31508004440C3D1FFF7A7FFFFF739FE0F4B1B6864338D
S315080044509842BAD9074B00221A70B6E7059B002B7B
S31508004460BFD101AB1B78FF2BBBD1079B022BB8D161
S31508004470FFF790FF29020020E801002078010020BC
S3150800448050010020670600002C0200202A020020A6
S31508004490002243088B4274D303098B425FD3030A75
S315080044A08B4244D3030B8B4228D3030C8B420DD388
S315080044B0FF22090212BA030C8B4202D31212090216
S315080044C065D0030B8B4219D300E0090AC30B8B4254
S315080044D001D3CB03C01A5241830B8B4201D38B0302
S315080044E0C01A5241430B8B4201D34B03C01A5241A7
S315080044F0030B8B4201D30B03C01A5241C30A8B42EA
S3150800450001D3CB02C01A5241830A8B4201D38B02D4
S31508004510C01A5241430A8B4201D34B02C01A524178
S31508004520030A8B4201D30B02C01A5241CDD2C309EA
S315080045308B4201D3CB01C01A524183098B4201D366
S315080045408B01C01A524143098B4201D34B01C01A51
S31508004550524103098B4201D30B01C01A5241C308C9
S315080045608B4201D3CB00C01A524183088B4201D338
S315080045708B00C01A524143088B4201D34B00C01A24
S315080045805241411A00D20146524110467047FFE790
S3150800459001B5002000F006F802BDC0460029F7D094
S315080045A076E770477047C046084B10B50400002BE5
S315080045B002D0002100E000BF054B1868836A002B73
S315080045C000D098472000FFF765FDC04600000000B0
S315080045D0A046000870B500260C4D0D4C641BA410AF
S315080045E0A64209D1002600F021F80A4D0A4C641BA0
S315080045F0A410A64205D170BDB300EB589847013602
S31508004600EEE7B300EB5898470136F2E7240100209D
S31508004610240100202401002028010020030012188C
S31508004620934200D1704719700133F9E7F8B5C046CF
S31508004630F8BC08BC9E467047F8B5C046F8BC08BC2E
S315080046409E467047000000000000000001020304B7
S315080046500607080900000000010203040203040516
S31508004660060708090A0B0C0D0E0F101001020304A9
S3150800467005060708090A0B0C0D0E0F10050206029F
S31508004680060307030803090309040A040B040C04B8
S315080046900C050D050E050F050F0610061007100868
S30D080046A0C40000200000000020
S30D080046A864E2FF7F0100000037
S315080046B000127A0000000000000000000000000060
S315080046C000000000000000000000000000000000DC
S315080046D000000000000000000000000000000000CC
S315080046E000000000000000000000000000000000BC
S315080046F000000000000000000000000000000000AC
S31508004700000000000000000000000000000000009B
S3110800471000000000ED280008C52800087D
S70508002800CA
